 rawmonitor

 Timestamp is a3722aa1 (reproducible build file hash)

 Preferred load address is 0000000180000000

 Start         Length     Name                   Class
 0001:00000000 00003230H .text$mn                CODE
 0001:00003230 00000036H .text$mn$00             CODE
 0001:00003266 00000092H .text$x                 CODE
 0002:00000000 00000198H .idata$5                DATA
 0002:00000198 00000038H .00cfg                  DATA
 0002:000001d0 00000008H .CRT$XCA                DATA
 0002:000001d8 00000008H .CRT$XCZ                DATA
 0002:000001e0 00000008H .CRT$XIA                DATA
 0002:000001e8 00000008H .CRT$XIC                DATA
 0002:000001f0 00000008H .CRT$XIZ                DATA
 0002:000001f8 00000008H .CRT$XLA                DATA
 0002:00000200 00000008H .CRT$XLZ                DATA
 0002:00000208 00000008H .CRT$XPA                DATA
 0002:00000210 00000008H .CRT$XPZ                DATA
 0002:00000218 00000008H .CRT$XTA                DATA
 0002:00000220 00000010H .CRT$XTZ                DATA
 0002:00000228 00000000H .gehcont$y              DATA
 0002:00000228 00000000H .gfids$y                DATA
 0002:00000230 00001d50H .rdata                  DATA
 0002:00001f80 00000000H .rdata$CastGuardVftablesA DATA
 0002:00001f80 00000000H .rdata$CastGuardVftablesC DATA
 0002:00001f80 00000028H .rdata$T                DATA
 0002:00001fa8 000000b8H .rdata$voltmd           DATA
 0002:00002060 00000318H .rdata$zzzdbg           DATA
 0002:00002378 00000008H .rtc$IAA                DATA
 0002:00002380 00000008H .rtc$IZZ                DATA
 0002:00002388 00000008H .rtc$TAA                DATA
 0002:00002390 00000008H .rtc$TZZ                DATA
 0002:00002398 00000004H .tls                    DATA
 0002:0000239c 00000004H .tls$                   DATA
 0002:000023a0 00000008H .tls$ZZZ                DATA
 0002:000023a8 00000308H .xdata                  DATA
 0002:000026b0 000004acH .edata                  DATA
 0002:00002b5c 00000064H .idata$2                DATA
 0002:00002bc0 00000018H .idata$3                DATA
 0002:00002bd8 00000198H .idata$4                DATA
 0002:00002d70 0000041eH .idata$6                DATA
 0003:00000000 00000080H .data                   DATA
 0003:00000080 0001b438H .bss                    DATA
 0004:00000000 000003d8H .pdata                  DATA

  Address         Publics by Value              Rva+Base               Lib:Object

 0000:00000000       __AbsoluteZero             0000000000000000     <absolute>
 0000:00000000       ___safe_se_handler_count   0000000000000000     <absolute>
 0000:00000000       ___safe_se_handler_table   0000000000000000     <absolute>
 0000:00000000       __arm64x_extra_rfe_table   0000000000000000     <absolute>
 0000:00000000       __arm64x_extra_rfe_table_size 0000000000000000     <absolute>
 0000:00000000       __arm64x_native_entrypoint 0000000000000000     <absolute>
 0000:00000000       __arm64x_redirection_metadata 0000000000000000     <absolute>
 0000:00000000       __arm64x_redirection_metadata_count 0000000000000000     <absolute>
 0000:00000000       __dynamic_value_reloc_table 0000000000000000     <absolute>
 0000:00000000       __enclave_config           0000000000000000     <absolute>
 0000:00000000       __guard_check_icall_a64n_fptr 0000000000000000     <absolute>
 0000:00000000       __guard_eh_cont_count      0000000000000000     <absolute>
 0000:00000000       __guard_eh_cont_table      0000000000000000     <absolute>
 0000:00000000       __guard_fids_count         0000000000000000     <absolute>
 0000:00000000       __guard_fids_table         0000000000000000     <absolute>
 0000:00000000       __guard_iat_count          0000000000000000     <absolute>
 0000:00000000       __guard_iat_table          0000000000000000     <absolute>
 0000:00000000       __guard_longjmp_count      0000000000000000     <absolute>
 0000:00000000       __guard_longjmp_table      0000000000000000     <absolute>
 0000:00000000       __hybrid_auxiliary_iat     0000000000000000     <absolute>
 0000:00000000       __hybrid_auxiliary_iat_copy 0000000000000000     <absolute>
 0000:00000000       __hybrid_code_map          0000000000000000     <absolute>
 0000:00000000       __hybrid_code_map_count    0000000000000000     <absolute>
 0000:00000000       __x64_code_ranges_to_entry_points 0000000000000000     <absolute>
 0000:00000000       __x64_code_ranges_to_entry_points_count 0000000000000000     <absolute>
 0000:00000100       __guard_flags              0000000000000100     <absolute>
 0000:00000000       __ImageBase                0000000180000000     <linker-defined>
 0001:00000000       ?NewObject@JNIEnv_@@QEAAPEAV_jobject@@PEAV_jclass@@PEAU_jmethodID@@ZZ 0000000180001000 f i librawmonitor.obj
 0001:00000024       ?SetEventNotificationMode@_jvmtiEnv@@QEAA?AW4jvmtiError@@W4jvmtiEventMode@@W4jvmtiEvent@@PEAV_jobject@@ZZ 0000000180001024 f i librawmonitor.obj
 0001:0000002c       ?TranslateError@@YAPEBDW4jvmtiError@@@Z 000000018000102c f   librawmonitor.obj
 0001:000002e4       ?nsk_jni_check_exception@@YAHPEAUJNIEnv_@@QEBDH@Z 00000001800012e4 f   librawmonitor.obj
 0001:00000428       ?nsk_jni_lverify@@YAHHPEAUJNIEnv_@@HQEBDH1ZZ 0000000180001428 f   librawmonitor.obj
 0001:000004c8       Agent_Initialize           00000001800014c8 f   librawmonitor.obj
 0001:000008b0       Agent_OnAttach             00000001800018b0 f   librawmonitor.obj
 0001:000008b0       Agent_OnLoad               00000001800018b0 f   librawmonitor.obj
 0001:000008b8       Java_nsk_jvmti_unit_FollowReferences_FollowRefObjects_addRefToVerify 00000001800018b8 f   librawmonitor.obj
 0001:00000a74       Java_nsk_jvmti_unit_FollowReferences_FollowRefObjects_getTag 0000000180001a74 f   librawmonitor.obj
 0001:00000b30       Java_nsk_jvmti_unit_FollowReferences_FollowRefObjects_resetRefsToVerify 0000000180001b30 f   librawmonitor.obj
 0001:00000b38       Java_nsk_jvmti_unit_FollowReferences_FollowRefObjects_resetTags 0000000180001b38 f   librawmonitor.obj
 0001:00000b7c       Java_nsk_jvmti_unit_FollowReferences_FollowRefObjects_setTag 0000000180001b7c f   librawmonitor.obj
 0001:00000dc8       Java_nsk_jvmti_unit_functions_rawmonitor_CreateRawMonitor 0000000180001dc8 f   librawmonitor.obj
 0001:00000e64       Java_nsk_jvmti_unit_functions_rawmonitor_GetResult 0000000180001e64 f   librawmonitor.obj
 0001:00000e6c       Java_nsk_jvmti_unit_functions_rawmonitor_RawMonitorEnter 0000000180001e6c f   librawmonitor.obj
 0001:00000ec0       Java_nsk_jvmti_unit_functions_rawmonitor_RawMonitorExit 0000000180001ec0 f   librawmonitor.obj
 0001:00000f14       Java_nsk_jvmti_unit_functions_rawmonitor_RawMonitorWait 0000000180001f14 f   librawmonitor.obj
 0001:00000f6c       Java_nsk_share_jvmti_ArgumentHandler_getAgentOptionsString 0000000180001f6c f   librawmonitor.obj
 0001:00001018       Java_nsk_share_jvmti_DebugeeClass_checkStatus 0000000180002018 f   librawmonitor.obj
 0001:000010a0       Java_nsk_share_jvmti_DebugeeClass_resetAgentData 00000001800020a0 f   librawmonitor.obj
 0001:00001100       Java_nsk_share_jvmti_RedefineAgent_agentStatus 0000000180002100 f   librawmonitor.obj
 0001:0000110c       Java_nsk_share_jvmti_RedefineAgent_isRedefined 000000018000210c f   librawmonitor.obj
 0001:00001118       Java_nsk_share_jvmti_RedefineAgent_redefineAttempted 0000000180002118 f   librawmonitor.obj
 0001:00001124       MA_checkStatus             0000000180002124 f   librawmonitor.obj
 0001:000011c8       __local_stdio_printf_options 00000001800021c8 f i librawmonitor.obj
 0001:000011d0       _snprintf                  00000001800021d0 f i librawmonitor.obj
 0001:000013f0       classFileLoadHookEvent     00000001800023f0 f   librawmonitor.obj
 0001:000015e4       debug_printf               00000001800025e4 f   librawmonitor.obj
 0001:00001640       exitOnError                0000000180002640 f   librawmonitor.obj
 0001:000016f4       fprintf                    00000001800026f4 f i librawmonitor.obj
 0001:00001738       init_callbacks             0000000180002738 f   librawmonitor.obj
 0001:00001790       nsk_jvmti_lverify          0000000180002790 f   librawmonitor.obj
 0001:00001880       nsk_jvmti_resetAgentData   0000000180002880 f   librawmonitor.obj
 0001:000018f4       nsk_lcomplain              00000001800028f4 f   librawmonitor.obj
 0001:00001914       nsk_ldisplay               0000000180002914 f   librawmonitor.obj
 0001:00001934       nsk_ltrace                 0000000180002934 f   librawmonitor.obj
 0001:00001954       nsk_lvcomplain             0000000180002954 f   librawmonitor.obj
 0001:00001b0c       nsk_lvdisplay              0000000180002b0c f   librawmonitor.obj
 0001:00001b58       nsk_lverify                0000000180002b58 f   librawmonitor.obj
 0001:00001bb4       nsk_lvtrace                0000000180002bb4 f   librawmonitor.obj
 0001:00001c14       nsk_printf                 0000000180002c14 f   librawmonitor.obj
 0001:00001c3c       nsk_vprintf                0000000180002c3c f   librawmonitor.obj
 0001:00001cf0       printf                     0000000180002cf0 f i librawmonitor.obj
 0001:000021f0       vmExit                     00000001800031f0 f   librawmonitor.obj
 0001:000021fc       vmInit                     00000001800031fc f   librawmonitor.obj
 0001:0000229c       vmStart                    000000018000329c f   librawmonitor.obj
 0001:00002308       __raise_securityfailure    0000000180003308 f   MSVCRT:gs_report.obj
 0001:0000233c       __report_gsfailure         000000018000333c f   MSVCRT:gs_report.obj
 0001:0000257c       __GSHandlerCheck           000000018000357c f   MSVCRT:gshandler.obj
 0001:0000259c       __GSHandlerCheckCommon     000000018000359c f   MSVCRT:gshandler.obj
 0001:00002610       __security_check_cookie    0000000180003610 f   MSVCRT:amdsecgs.obj
 0001:00002950       _DllMainCRTStartup         0000000180003950 f   MSVCRT:dll_dllmain.obj
 0001:00002990       __scrt_acquire_startup_lock 0000000180003990 f   MSVCRT:utility.obj
 0001:000029cc       __scrt_dllmain_after_initialize_c 00000001800039cc f   MSVCRT:utility.obj
 0001:00002a00       __scrt_dllmain_before_initialize_c 0000000180003a00 f   MSVCRT:utility.obj
 0001:00002a18       __scrt_dllmain_crt_thread_attach 0000000180003a18 f   MSVCRT:utility.obj
 0001:00002a40       __scrt_dllmain_crt_thread_detach 0000000180003a40 f   MSVCRT:utility.obj
 0001:00002a58       __scrt_dllmain_exception_filter 0000000180003a58 f   MSVCRT:utility.obj
 0001:00002ab8       __scrt_dllmain_uninitialize_c 0000000180003ab8 f   MSVCRT:utility.obj
 0001:00002ae8       __scrt_dllmain_uninitialize_critical 0000000180003ae8 f   MSVCRT:utility.obj
 0001:00002afc       __scrt_initialize_crt      0000000180003afc f   MSVCRT:utility.obj
 0001:00002b48       __scrt_initialize_onexit_tables 0000000180003b48 f   MSVCRT:utility.obj
 0001:00002bd4       __scrt_is_nonwritable_in_current_image 0000000180003bd4 f   MSVCRT:utility.obj
 0001:00002c6c       __scrt_release_startup_lock 0000000180003c6c f   MSVCRT:utility.obj
 0001:00002c90       __scrt_uninitialize_crt    0000000180003c90 f   MSVCRT:utility.obj
 0001:00002cbc       _onexit                    0000000180003cbc f   MSVCRT:utility.obj
 0001:00002cf8       atexit                     0000000180003cf8 f   MSVCRT:utility.obj
 0001:00002d10       __crt_debugger_hook        0000000180003d10 f   MSVCRT:utility_desktop.obj
 0001:00002d18       __scrt_fastfail            0000000180003d18 f   MSVCRT:utility_desktop.obj
 0001:00002e64       _guard_check_icall_nop     0000000180003e64 f i MSVCRT:guard_support.obj
 0001:00002e68       __security_init_cookie     0000000180003e68 f   MSVCRT:gs_support.obj
 0001:00002f14       DllMain                    0000000180003f14 f   MSVCRT:dll_dllmain_stub.obj
 0001:00002f38       ?__scrt_initialize_type_info@@YAXXZ 0000000180003f38 f   MSVCRT:tncleanup.obj
 0001:00002f48       ?__scrt_uninitialize_type_info@@YAXXZ 0000000180003f48 f   MSVCRT:tncleanup.obj
 0001:00002f54       __local_stdio_scanf_options 0000000180003f54 f i MSVCRT:default_local_stdio_options.obj
 0001:00002f5c       __scrt_initialize_default_local_stdio_options 0000000180003f5c f   MSVCRT:default_local_stdio_options.obj
 0001:00002f78       __scrt_get_dyn_tls_init_callback 0000000180003f78 f   MSVCRT:dyn_tls_init.obj
 0001:00002f80       _RTC_Initialize            0000000180003f80 f   MSVCRT:initsect.obj
 0001:00002fbc       _RTC_Terminate             0000000180003fbc f   MSVCRT:initsect.obj
 0001:00002ff8       __isa_available_init       0000000180003ff8 f   MSVCRT:cpu_disp.obj
 0001:000031a4       _get_startup_argv_mode     00000001800041a4 f   MSVCRT:argv_mode.obj
 0001:000031ac       __scrt_is_ucrt_dll_in_use  00000001800041ac f   MSVCRT:ucrt_detection.obj
 0001:000031c0       memcpy                     00000001800041c0 f   vcruntime:VCRUNTIME140.dll
 0001:000031c6       memset                     00000001800041c6 f   vcruntime:VCRUNTIME140.dll
 0001:000031cc       strchr                     00000001800041cc f   vcruntime:VCRUNTIME140.dll
 0001:000031d2       strstr                     00000001800041d2 f   vcruntime:VCRUNTIME140.dll
 0001:000031d8       __C_specific_handler       00000001800041d8 f   vcruntime:VCRUNTIME140.dll
 0001:000031de       __std_type_info_destroy_list 00000001800041de f   vcruntime:VCRUNTIME140.dll
 0001:000031e4       strlen                     00000001800041e4 f   ucrt:api-ms-win-crt-string-l1-1-0.dll
 0001:000031ea       _initterm                  00000001800041ea f   ucrt:api-ms-win-crt-runtime-l1-1-0.dll
 0001:000031f0       _initterm_e                00000001800041f0 f   ucrt:api-ms-win-crt-runtime-l1-1-0.dll
 0001:000031f6       _seh_filter_dll            00000001800041f6 f   ucrt:api-ms-win-crt-runtime-l1-1-0.dll
 0001:000031fc       _configure_narrow_argv     00000001800041fc f   ucrt:api-ms-win-crt-runtime-l1-1-0.dll
 0001:00003202       _initialize_narrow_environment 0000000180004202 f   ucrt:api-ms-win-crt-runtime-l1-1-0.dll
 0001:00003208       _initialize_onexit_table   0000000180004208 f   ucrt:api-ms-win-crt-runtime-l1-1-0.dll
 0001:0000320e       _register_onexit_function  000000018000420e f   ucrt:api-ms-win-crt-runtime-l1-1-0.dll
 0001:00003214       _execute_onexit_table      0000000180004214 f   ucrt:api-ms-win-crt-runtime-l1-1-0.dll
 0001:0000321a       _crt_atexit                000000018000421a f   ucrt:api-ms-win-crt-runtime-l1-1-0.dll
 0001:00003220       _cexit                     0000000180004220 f   ucrt:api-ms-win-crt-runtime-l1-1-0.dll
 0001:00003228       __acrt_initialize          0000000180004228 f   MSVCRT:ucrt_stubs.obj
 0001:00003228       __acrt_thread_attach       0000000180004228 f   MSVCRT:ucrt_stubs.obj
 0001:00003228       __acrt_thread_detach       0000000180004228 f   MSVCRT:ucrt_stubs.obj
 0001:00003228       __acrt_uninitialize        0000000180004228 f   MSVCRT:ucrt_stubs.obj
 0001:00003228       __acrt_uninitialize_critical 0000000180004228 f   MSVCRT:ucrt_stubs.obj
 0001:00003228       __scrt_stub_for_acrt_initialize 0000000180004228 f   MSVCRT:ucrt_stubs.obj
 0001:00003228       __scrt_stub_for_acrt_thread_attach 0000000180004228 f   MSVCRT:ucrt_stubs.obj
 0001:00003228       __scrt_stub_for_acrt_thread_detach 0000000180004228 f   MSVCRT:ucrt_stubs.obj
 0001:00003228       __scrt_stub_for_acrt_uninitialize 0000000180004228 f   MSVCRT:ucrt_stubs.obj
 0001:00003228       __scrt_stub_for_acrt_uninitialize_critical 0000000180004228 f   MSVCRT:ucrt_stubs.obj
 0001:00003228       __vcrt_initialize          0000000180004228 f   MSVCRT:ucrt_stubs.obj
 0001:00003228       __vcrt_thread_attach       0000000180004228 f   MSVCRT:ucrt_stubs.obj
 0001:00003228       __vcrt_thread_detach       0000000180004228 f   MSVCRT:ucrt_stubs.obj
 0001:00003228       __vcrt_uninitialize        0000000180004228 f   MSVCRT:ucrt_stubs.obj
 0001:00003228       __vcrt_uninitialize_critical 0000000180004228 f   MSVCRT:ucrt_stubs.obj
 0001:0000322c       __scrt_stub_for_is_c_termination_complete 000000018000422c f   MSVCRT:ucrt_stubs.obj
 0001:0000322c       _is_c_termination_complete 000000018000422c f   MSVCRT:ucrt_stubs.obj
 0001:00003240       _guard_dispatch_icall_nop  0000000180004240 f   MSVCRT:guard_dispatch.obj
 0001:00003260       _guard_xfg_dispatch_icall_nop 0000000180004260 f   MSVCRT:guard_xfg_dispatch.obj
 0002:00000000       __imp_RtlCaptureContext    0000000180005000     kernel32:KERNEL32.dll
 0002:00000008       __imp_RtlLookupFunctionEntry 0000000180005008     kernel32:KERNEL32.dll
 0002:00000010       __imp_RtlVirtualUnwind     0000000180005010     kernel32:KERNEL32.dll
 0002:00000018       __imp_UnhandledExceptionFilter 0000000180005018     kernel32:KERNEL32.dll
 0002:00000020       __imp_SetUnhandledExceptionFilter 0000000180005020     kernel32:KERNEL32.dll
 0002:00000028       __imp_GetCurrentProcess    0000000180005028     kernel32:KERNEL32.dll
 0002:00000030       __imp_TerminateProcess     0000000180005030     kernel32:KERNEL32.dll
 0002:00000038       __imp_IsProcessorFeaturePresent 0000000180005038     kernel32:KERNEL32.dll
 0002:00000040       __imp_CloseHandle          0000000180005040     kernel32:KERNEL32.dll
 0002:00000048       __imp_InitializeCriticalSectionAndSpinCount 0000000180005048     kernel32:KERNEL32.dll
 0002:00000050       __imp_DeleteCriticalSection 0000000180005050     kernel32:KERNEL32.dll
 0002:00000058       __imp_CreateEventW         0000000180005058     kernel32:KERNEL32.dll
 0002:00000060       __imp_GetModuleHandleW     0000000180005060     kernel32:KERNEL32.dll
 0002:00000068       __imp_GetProcAddress       0000000180005068     kernel32:KERNEL32.dll
 0002:00000070       __imp_IsDebuggerPresent    0000000180005070     kernel32:KERNEL32.dll
 0002:00000078       __imp_QueryPerformanceCounter 0000000180005078     kernel32:KERNEL32.dll
 0002:00000080       __imp_GetCurrentProcessId  0000000180005080     kernel32:KERNEL32.dll
 0002:00000088       __imp_GetCurrentThreadId   0000000180005088     kernel32:KERNEL32.dll
 0002:00000090       __imp_GetSystemTimeAsFileTime 0000000180005090     kernel32:KERNEL32.dll
 0002:00000098       __imp_DisableThreadLibraryCalls 0000000180005098     kernel32:KERNEL32.dll
 0002:000000a0       __imp_InitializeSListHead  00000001800050a0     kernel32:KERNEL32.dll
 0002:000000a8       \177KERNEL32_NULL_THUNK_DATA 00000001800050a8     kernel32:KERNEL32.dll
 0002:000000b0       __imp_memcpy               00000001800050b0     vcruntime:VCRUNTIME140.dll
 0002:000000b8       __imp_memset               00000001800050b8     vcruntime:VCRUNTIME140.dll
 0002:000000c0       __imp_strchr               00000001800050c0     vcruntime:VCRUNTIME140.dll
 0002:000000c8       __imp_strstr               00000001800050c8     vcruntime:VCRUNTIME140.dll
 0002:000000d0       __imp___C_specific_handler 00000001800050d0     vcruntime:VCRUNTIME140.dll
 0002:000000d8       __imp___std_type_info_destroy_list 00000001800050d8     vcruntime:VCRUNTIME140.dll
 0002:000000e0       \177VCRUNTIME140_NULL_THUNK_DATA 00000001800050e0     vcruntime:VCRUNTIME140.dll
 0002:000000e8       __imp__errno               00000001800050e8     ucrt:api-ms-win-crt-runtime-l1-1-0.dll
 0002:000000f0       __imp_exit                 00000001800050f0     ucrt:api-ms-win-crt-runtime-l1-1-0.dll
 0002:000000f8       __imp__cexit               00000001800050f8     ucrt:api-ms-win-crt-runtime-l1-1-0.dll
 0002:00000100       __imp__crt_atexit          0000000180005100     ucrt:api-ms-win-crt-runtime-l1-1-0.dll
 0002:00000108       __imp__execute_onexit_table 0000000180005108     ucrt:api-ms-win-crt-runtime-l1-1-0.dll
 0002:00000110       __imp__register_onexit_function 0000000180005110     ucrt:api-ms-win-crt-runtime-l1-1-0.dll
 0002:00000118       __imp__initialize_onexit_table 0000000180005118     ucrt:api-ms-win-crt-runtime-l1-1-0.dll
 0002:00000120       __imp__initialize_narrow_environment 0000000180005120     ucrt:api-ms-win-crt-runtime-l1-1-0.dll
 0002:00000128       __imp__configure_narrow_argv 0000000180005128     ucrt:api-ms-win-crt-runtime-l1-1-0.dll
 0002:00000130       __imp__seh_filter_dll      0000000180005130     ucrt:api-ms-win-crt-runtime-l1-1-0.dll
 0002:00000138       __imp__initterm_e          0000000180005138     ucrt:api-ms-win-crt-runtime-l1-1-0.dll
 0002:00000140       __imp__initterm            0000000180005140     ucrt:api-ms-win-crt-runtime-l1-1-0.dll
 0002:00000148       \177api-ms-win-crt-runtime-l1-1-0_NULL_THUNK_DATA 0000000180005148     ucrt:api-ms-win-crt-runtime-l1-1-0.dll
 0002:00000150       __imp___acrt_iob_func      0000000180005150     ucrt:api-ms-win-crt-stdio-l1-1-0.dll
 0002:00000158       __imp_fflush               0000000180005158     ucrt:api-ms-win-crt-stdio-l1-1-0.dll
 0002:00000160       __imp___stdio_common_vsprintf 0000000180005160     ucrt:api-ms-win-crt-stdio-l1-1-0.dll
 0002:00000168       __imp___stdio_common_vfprintf 0000000180005168     ucrt:api-ms-win-crt-stdio-l1-1-0.dll
 0002:00000170       \177api-ms-win-crt-stdio-l1-1-0_NULL_THUNK_DATA 0000000180005170     ucrt:api-ms-win-crt-stdio-l1-1-0.dll
 0002:00000178       __imp__strdup              0000000180005178     ucrt:api-ms-win-crt-string-l1-1-0.dll
 0002:00000178       __imp_strdup               0000000180005178     ucrt:api-ms-win-crt-string-l1-1-0.dll
 0002:00000180       __imp_strlen               0000000180005180     ucrt:api-ms-win-crt-string-l1-1-0.dll
 0002:00000188       __imp_strncpy              0000000180005188     ucrt:api-ms-win-crt-string-l1-1-0.dll
 0002:00000190       \177api-ms-win-crt-string-l1-1-0_NULL_THUNK_DATA 0000000180005190     ucrt:api-ms-win-crt-string-l1-1-0.dll
 0002:00000198       __guard_check_icall_fptr   0000000180005198     MSVCRT:guard_support.obj
 0002:000001a0       __guard_xfg_check_icall_fptr 00000001800051a0     MSVCRT:guard_support.obj
 0002:000001a8       __guard_dispatch_icall_fptr 00000001800051a8     MSVCRT:guard_support.obj
 0002:000001b0       __guard_xfg_dispatch_icall_fptr 00000001800051b0     MSVCRT:guard_support.obj
 0002:000001b8       __guard_xfg_table_dispatch_icall_fptr 00000001800051b8     MSVCRT:guard_support.obj
 0002:000001c0       __castguard_check_failure_os_handled_fptr 00000001800051c0     MSVCRT:guard_support.obj
 0002:000001c8       __guard_memcpy_fptr        00000001800051c8     vcruntime:softmemtag.obj
 0002:000001d0       __xc_a                     00000001800051d0     MSVCRT:initializers.obj
 0002:000001d8       __xc_z                     00000001800051d8     MSVCRT:initializers.obj
 0002:000001e0       __xi_a                     00000001800051e0     MSVCRT:initializers.obj
 0002:000001f0       __xi_z                     00000001800051f0     MSVCRT:initializers.obj
 0002:000001f8       __xl_a                     00000001800051f8     MSVCRT:tlssup.obj
 0002:00000200       __xl_z                     0000000180005200     MSVCRT:tlssup.obj
 0002:00000208       __xp_a                     0000000180005208     MSVCRT:initializers.obj
 0002:00000210       __xp_z                     0000000180005210     MSVCRT:initializers.obj
 0002:00000218       __xt_a                     0000000180005218     MSVCRT:initializers.obj
 0002:00000220       __xt_z                     0000000180005220     MSVCRT:initializers.obj
 0002:00000230       g_refKindStr               0000000180005230     librawmonitor.obj
 0002:000003e0       ??_C@_09BPLDFGCI@unknown_0@ 00000001800053e0     librawmonitor.obj
 0002:000003f0       ??_C@_0BL@FPNMECJD@JVMTI_HEAP_REFERENCE_CLASS@ 00000001800053f0     librawmonitor.obj
 0002:00000410       ??_C@_0BL@FKGKKLNM@JVMTI_HEAP_REFERENCE_FIELD@ 0000000180005410     librawmonitor.obj
 0002:00000430       ??_C@_0CD@CAEHCFJF@JVMTI_HEAP_REFERENCE_ARRAY_ELEM@ 0000000180005430     librawmonitor.obj
 0002:00000458       ??_C@_0CC@DNEBMCNK@JVMTI_HEAP_REFERENCE_CLASS_LOAD@ 0000000180005458     librawmonitor.obj
 0002:00000480       ??_C@_0BN@CJMIPEBB@JVMTI_HEAP_REFERENCE_SIGNERS@ 0000000180005480     librawmonitor.obj
 0002:000004a0       ??_C@_0CH@HBOIDPEB@JVMTI_HEAP_REFERENCE_PROTECTION@ 00000001800054a0     librawmonitor.obj
 0002:000004c8       ??_C@_0BP@MDKGDGKL@JVMTI_HEAP_REFERENCE_INTERFACE@ 00000001800054c8     librawmonitor.obj
 0002:000004e8       ??_C@_0CC@JJMIHNJH@JVMTI_HEAP_REFERENCE_STATIC_FIE@ 00000001800054e8     librawmonitor.obj
 0002:00000510       ??_C@_0CD@IDHEEGID@JVMTI_HEAP_REFERENCE_CONSTANT_P@ 0000000180005510     librawmonitor.obj
 0002:00000538       ??_C@_0CA@EFFCHNG@JVMTI_HEAP_REFERENCE_SUPERCLASS@ 0000000180005538     librawmonitor.obj
 0002:00000558       ??_C@_0L@PCDFHGCJ@unknown_11@ 0000000180005558     librawmonitor.obj
 0002:00000568       ??_C@_0L@NJBICFOK@unknown_12@ 0000000180005568     librawmonitor.obj
 0002:00000578       ??_C@_0L@MAADBEKL@unknown_13@ 0000000180005578     librawmonitor.obj
 0002:00000588       ??_C@_0L@IPECICGM@unknown_14@ 0000000180005588     librawmonitor.obj
 0002:00000598       ??_C@_0L@JGFJLDCN@unknown_15@ 0000000180005598     librawmonitor.obj
 0002:000005a8       ??_C@_0L@LNHEOAOO@unknown_16@ 00000001800055a8     librawmonitor.obj
 0002:000005b8       ??_C@_0L@KEGPNBKP@unknown_17@ 00000001800055b8     librawmonitor.obj
 0002:000005c8       ??_C@_0L@CDPHMNGA@unknown_18@ 00000001800055c8     librawmonitor.obj
 0002:000005d8       ??_C@_0L@DKOMPMCB@unknown_19@ 00000001800055d8     librawmonitor.obj
 0002:000005e8       ??_C@_0L@OJGIPJDB@unknown_20@ 00000001800055e8     librawmonitor.obj
 0002:000005f8       ??_C@_0CA@KAOFNDEM@JVMTI_HEAP_REFERENCE_JNI_GLOBAL@ 00000001800055f8     librawmonitor.obj
 0002:00000618       ??_C@_0CC@HPFAJBK@JVMTI_HEAP_REFERENCE_SYSTEM_CLA@ 0000000180005618     librawmonitor.obj
 0002:00000640       ??_C@_0BN@FDEGFOHC@JVMTI_HEAP_REFERENCE_MONITOR@ 0000000180005640     librawmonitor.obj
 0002:00000660       ??_C@_0CB@HKIBCMAJ@JVMTI_HEAP_REFERENCE_STACK_LOCA@ 0000000180005660     librawmonitor.obj
 0002:00000688       ??_C@_0BP@EAACMMOE@JVMTI_HEAP_REFERENCE_JNI_LOCAL@ 0000000180005688     librawmonitor.obj
 0002:000006a8       ??_C@_0BM@IJDEOGOE@JVMTI_HEAP_REFERENCE_THREAD@ 00000001800056a8     librawmonitor.obj
 0002:000006c8       ??_C@_0BL@EDGPPKC@JVMTI_HEAP_REFERENCE_OTHER@ 00000001800056c8     librawmonitor.obj
 0002:000006e4       ??_C@_04BCJPDBDA@Code@     00000001800056e4     librawmonitor.obj
 0002:000006f0       ??_C@_0BA@OCLMCFKC@LineNumberTable@ 00000001800056f0     librawmonitor.obj
 0002:00000700       ??_C@_0BD@CPAEPILC@LocalVariableTable@ 0000000180005700     librawmonitor.obj
 0002:00000718       ??_C@_0BH@NMBDNHBD@LocalVariableTypeTable@ 0000000180005718     librawmonitor.obj
 0002:00000730       ??_C@_0O@HIHEEDNJ@StackMapTable@ 0000000180005730     librawmonitor.obj
 0002:00000740       ??_C@_0L@HCDIAMJG@?9?5?$CFs?0?5?$CFd?3?5@ 0000000180005740     librawmonitor.obj
 0002:00000750       ??_C@_0JI@HLPECLFI@?$CD?5?4?4?4?6?$CD?5ERROR?3?5too?5many?5complai@ 0000000180005750     librawmonitor.obj
 0002:000007f0       ??_C@_0ED@JNEKCCOB@The?5following?5fake?5exception?5st@ 00000001800057f0     librawmonitor.obj
 0002:00000838       ??_C@_0CN@FCNMDFBH@nsk?4share?4Fake_Exception_for_RU@ 0000000180005838     librawmonitor.obj
 0002:00000868       ??_C@_08PGFFNAEI@?$CI?$CFs?3?$CFd?$CJ?5@ 0000000180005868     librawmonitor.obj
 0002:00000878       ??_C@_0DP@IENMAEGI@s?2test?2hotspot?2jtreg?2vmTestbase@ 0000000180005878     librawmonitor.obj
 0002:000008b8       ??_C@_0BL@NDJLFFJB@?7at?5nsk_lvcomplain?$CI?$CFs?3?$CFd?$CJ?6@ 00000001800058b8     librawmonitor.obj
 0002:000008d8       ??_C@_0BC@JOOKAFKF@?$CD?5ERROR?3?5?$CFs?0?5?$CFd?3?5@ 00000001800058d8     librawmonitor.obj
 0002:000008f0       ??_C@_09KJEAHMEH@?$CD?5ERROR?3?5@ 00000001800058f0     librawmonitor.obj
 0002:000008fc       ??_C@_02GPIOPFAK@?$DO?$DO@ 00000001800058fc     librawmonitor.obj
 0002:00000900       ??_C@_02FODMEDOG@?$DM?$DM@ 0000000180005900     librawmonitor.obj
 0002:00000904       ??_C@_02DJGKEECL@?4?4@     0000000180005904     librawmonitor.obj
 0002:00000908       ??_C@_0O@CJPGJOAF@?9?5?$CFs?0?5?$CFd?3?5?$CFs?5@ 0000000180005908     librawmonitor.obj
 0002:00000918       ??_C@_0CB@IAKPDOIC@?$CD?5?5?5verified?5assertion?5is?5FALSE@ 0000000180005918     librawmonitor.obj
 0002:00000940       ??_C@_0CO@LGONDEPD@stdout?3?5fflush?5failed?5?9?5err?$DN?$CFd?5@ 0000000180005940     librawmonitor.obj
 0002:00000970       ??_C@_0CO@KBGKJPBD@stderr?3?5fflush?5failed?5?9?5err?$DN?$CFd?5@ 0000000180005970     librawmonitor.obj
 0002:000009a0       ??_C@_0BB@JCNMKLLK@JVMTI_ERROR_NONE@ 00000001800059a0     librawmonitor.obj
 0002:000009b8       ??_C@_0BL@LDIMKLPH@JVMTI_ERROR_INVALID_THREAD@ 00000001800059b8     librawmonitor.obj
 0002:000009d8       ??_C@_0CB@PJFPAIKJ@JVMTI_ERROR_INVALID_THREAD_GROU@ 00000001800059d8     librawmonitor.obj
 0002:00000a00       ??_C@_0BN@LLMKHMNF@JVMTI_ERROR_INVALID_PRIORITY@ 0000000180005a00     librawmonitor.obj
 0002:00000a20       ??_C@_0CB@MBOFKAGB@JVMTI_ERROR_THREAD_NOT_SUSPENDE@ 0000000180005a20     librawmonitor.obj
 0002:00000a48       ??_C@_0BN@FABOLPBI@JVMTI_ERROR_THREAD_SUSPENDED@ 0000000180005a48     librawmonitor.obj
 0002:00000a68       ??_C@_0BN@FDGNOBJM@JVMTI_ERROR_THREAD_NOT_ALIVE@ 0000000180005a68     librawmonitor.obj
 0002:00000a88       ??_C@_0BL@GOBIFKNJ@JVMTI_ERROR_INVALID_OBJECT@ 0000000180005a88     librawmonitor.obj
 0002:00000aa8       ??_C@_0BK@FCMAJPPC@JVMTI_ERROR_INVALID_CLASS@ 0000000180005aa8     librawmonitor.obj
 0002:00000ac8       ??_C@_0BP@IKLLBKEB@JVMTI_ERROR_CLASS_NOT_PREPARED@ 0000000180005ac8     librawmonitor.obj
 0002:00000ae8       ??_C@_0BN@KLPPLKG@JVMTI_ERROR_INVALID_METHODID@ 0000000180005ae8     librawmonitor.obj
 0002:00000b08       ??_C@_0BN@BCEKOKND@JVMTI_ERROR_INVALID_LOCATION@ 0000000180005b08     librawmonitor.obj
 0002:00000b28       ??_C@_0BM@DFDGPME@JVMTI_ERROR_INVALID_FIELDID@ 0000000180005b28     librawmonitor.obj
 0002:00000b48       ??_C@_0BL@NELIEPEC@JVMTI_ERROR_NO_MORE_FRAMES@ 0000000180005b48     librawmonitor.obj
 0002:00000b68       ??_C@_0BJ@BDBECFDM@JVMTI_ERROR_OPAQUE_FRAME@ 0000000180005b68     librawmonitor.obj
 0002:00000b88       ??_C@_0BK@MIIFNLOB@JVMTI_ERROR_TYPE_MISMATCH@ 0000000180005b88     librawmonitor.obj
 0002:00000ba8       ??_C@_0BJ@HPCAOILC@JVMTI_ERROR_INVALID_SLOT@ 0000000180005ba8     librawmonitor.obj
 0002:00000bc8       ??_C@_0BG@CHILOPNI@JVMTI_ERROR_DUPLICATE@ 0000000180005bc8     librawmonitor.obj
 0002:00000be0       ??_C@_0BG@DIEMLHKM@JVMTI_ERROR_NOT_FOUND@ 0000000180005be0     librawmonitor.obj
 0002:00000bf8       ??_C@_0BM@NHMCKHOB@JVMTI_ERROR_INVALID_MONITOR@ 0000000180005bf8     librawmonitor.obj
 0002:00000c18       ??_C@_0BO@PPEDAJGL@JVMTI_ERROR_NOT_MONITOR_OWNER@ 0000000180005c18     librawmonitor.obj
 0002:00000c38       ??_C@_0BG@FCAIPEID@JVMTI_ERROR_INTERRUPT@ 0000000180005c38     librawmonitor.obj
 0002:00000c50       ??_C@_0CB@EGDBNKOI@JVMTI_ERROR_INVALID_CLASS_FORMA@ 0000000180005c50     librawmonitor.obj
 0002:00000c78       ??_C@_0CG@DGKOGIAL@JVMTI_ERROR_CIRCULAR_CLASS_DEFI@ 0000000180005c78     librawmonitor.obj
 0002:00000ca0       ??_C@_0BP@ICEALPKC@JVMTI_ERROR_FAILS_VERIFICATION@ 0000000180005ca0     librawmonitor.obj
 0002:00000cc0       ??_C@_0DC@JDACLMIO@JVMTI_ERROR_UNSUPPORTED_REDEFIN@ 0000000180005cc0     librawmonitor.obj
 0002:00000cf8       ??_C@_0DE@GKDKNOMJ@JVMTI_ERROR_UNSUPPORTED_REDEFIN@ 0000000180005cf8     librawmonitor.obj
 0002:00000d30       ??_C@_0BO@LAFKIOG@JVMTI_ERROR_INVALID_TYPESTATE@ 0000000180005d30     librawmonitor.obj
 0002:00000d50       ??_C@_0DH@INDGCLLB@JVMTI_ERROR_UNSUPPORTED_REDEFIN@ 0000000180005d50     librawmonitor.obj
 0002:00000d88       ??_C@_0DE@NHEOMMGI@JVMTI_ERROR_UNSUPPORTED_REDEFIN@ 0000000180005d88     librawmonitor.obj
 0002:00000dc0       ??_C@_0CA@EKPNJOEP@JVMTI_ERROR_UNSUPPORTED_VERSION@ 0000000180005dc0     librawmonitor.obj
 0002:00000de0       ??_C@_0BN@OFFMAHHL@JVMTI_ERROR_NAMES_DONT_MATCH@ 0000000180005de0     librawmonitor.obj
 0002:00000e00       ??_C@_0DN@HHBBLAKE@JVMTI_ERROR_UNSUPPORTED_REDEFIN@ 0000000180005e00     librawmonitor.obj
 0002:00000e40       ??_C@_0DO@HMBGBGNA@JVMTI_ERROR_UNSUPPORTED_REDEFIN@ 0000000180005e40     librawmonitor.obj
 0002:00000e80       ??_C@_0BP@PBECGKHJ@JVMTI_ERROR_UNMODIFIABLE_CLASS@ 0000000180005e80     librawmonitor.obj
 0002:00000ea0       ??_C@_0BK@CANILEHF@JVMTI_ERROR_NOT_AVAILABLE@ 0000000180005ea0     librawmonitor.obj
 0002:00000ec0       ??_C@_0CE@INJKMEFK@JVMTI_ERROR_MUST_POSSESS_CAPABI@ 0000000180005ec0     librawmonitor.obj
 0002:00000ee8       ??_C@_0BJ@LBFPFPDM@JVMTI_ERROR_NULL_POINTER@ 0000000180005ee8     librawmonitor.obj
 0002:00000f08       ??_C@_0BP@CHJPNNEM@JVMTI_ERROR_ABSENT_INFORMATION@ 0000000180005f08     librawmonitor.obj
 0002:00000f28       ??_C@_0BP@OMFMNLC@JVMTI_ERROR_INVALID_EVENT_TYPE@ 0000000180005f28     librawmonitor.obj
 0002:00000f48       ??_C@_0BN@BIBNPHHO@JVMTI_ERROR_ILLEGAL_ARGUMENT@ 0000000180005f48     librawmonitor.obj
 0002:00000f68       ??_C@_0BK@KKNDHDCE@JVMTI_ERROR_NATIVE_METHOD@ 0000000180005f68     librawmonitor.obj
 0002:00000f88       ??_C@_0BK@PMKCFHAE@JVMTI_ERROR_OUT_OF_MEMORY@ 0000000180005f88     librawmonitor.obj
 0002:00000fa8       ??_C@_0BK@NNJBDMNB@JVMTI_ERROR_ACCESS_DENIED@ 0000000180005fa8     librawmonitor.obj
 0002:00000fc8       ??_C@_0BI@GHECLMNC@JVMTI_ERROR_WRONG_PHASE@ 0000000180005fc8     librawmonitor.obj
 0002:00000fe0       ??_C@_0BF@OLIHJOII@JVMTI_ERROR_INTERNAL@ 0000000180005fe0     librawmonitor.obj
 0002:00000ff8       ??_C@_0BO@EOHGKJHI@JVMTI_ERROR_UNATTACHED_THREAD@ 0000000180005ff8     librawmonitor.obj
 0002:00001018       ??_C@_0CA@LKHFDACL@JVMTI_ERROR_INVALID_ENVIRONMENT@ 0000000180006018     librawmonitor.obj
 0002:00001038       ??_C@_0BA@MMFHLOKK@?$DMunknown?5error?$DO@ 0000000180006038     librawmonitor.obj
 0002:00001048       ??_C@_0CF@CBHOKDB@throwable?5?$DN?5jni?9?$DOExceptionOccur@ 0000000180006048     librawmonitor.obj
 0002:00001070       ??_C@_03OFAPEBGM@?$CFs?6@  0000000180006070     librawmonitor.obj
 0002:00001078       ??_C@_0DM@LPIGEGNJ@s?2test?2hotspot?2jtreg?2vmTestbase@ 0000000180006078     librawmonitor.obj
 0002:000010b8       ??_C@_0CC@NFCNPEPK@Exception?5in?5JNI?5call?5?$CIcleared?$CJ@ 00000001800060b8     librawmonitor.obj
 0002:000010e0       ??_C@_0BJ@IBAKFIKF@jni?9?$DOExceptionDescribe?$CI?$CJ@ 00000001800060e0     librawmonitor.obj
 0002:00001100       ??_C@_0BG@GGKALKMH@jni?9?$DOExceptionClear?$CI?$CJ@ 0000000180006100     librawmonitor.obj
 0002:00001118       ??_C@_0CF@JMGFGJLJ@?$CD?5?5?5verified?5JNI?5assertion?5is?5F@ 0000000180006118     librawmonitor.obj
 0002:00001140       ??_C@_0CB@MLNJNCLJ@?5?5jvmti?5error?3?5code?$DN?$CFd?0?5name?$DN?$CFs@ 0000000180006140     librawmonitor.obj
 0002:00001168       ??_C@_0CD@OHBGDKMK@?$CD?5?5?5jvmti?5error?3?5code?$DN?$CFd?0?5name?$DN@ 0000000180006168     librawmonitor.obj
 0002:00001190       ??_C@_0CG@JNNCGPHB@?$CD?5?5?5error?5expected?3?5code?$DN?$CFd?0?5na@ 0000000180006190     librawmonitor.obj
 0002:000011c0       ??_C@_0EB@IMGKPCGE@?$CIstr_obj?5?$DN?5jni?9?$DONewStringUTF?$CIco@ 00000001800061c0     librawmonitor.obj
 0002:00001210       ??_C@_0EA@HFOGGBCC@s?2test?2hotspot?2jtreg?2vmTestbase@ 0000000180006210     librawmonitor.obj
 0002:00001250       ??_C@_05KKCIMGE@error@     0000000180006250     librawmonitor.obj
 0002:00001260       ??_C@_0EA@PNBCDMOA@s?2test?2hotspot?2jtreg?2vmTestbase@ 0000000180006260     librawmonitor.obj
 0002:000012a0       ??_C@_0DI@ILAHDLMP@?$CI?$CKagentThreadProc?$CJ?$CIjvmti_env?0?5a@ 00000001800062a0     librawmonitor.obj
 0002:000012d8       ??_C@_0BD@KDBALNLB@JVMTI?5agent?5thread@ 00000001800062d8     librawmonitor.obj
 0002:000012f0       ??_C@_0BB@NOKBFPFO@java?1lang?1Thread@ 00000001800062f0     librawmonitor.obj
 0002:00001304       ??_C@_06FALKBLGB@?$DMinit?$DO@ 0000000180006304     librawmonitor.obj
 0002:00001310       ??_C@_0BG@IKDDPPGD@?$CILjava?1lang?1String?$DL?$CJV@ 0000000180006310     librawmonitor.obj
 0002:00001330       ??_C@_0EB@IFJBFEKC@?$CIthreadClass?5?$DN?5jni_env?9?$DOFindCla@ 0000000180006330     librawmonitor.obj
 0002:00001380       ??_C@_0GF@FGFIBKKL@?$CIthreadCtor?5?$DN?5jni_env?9?$DOGetMetho@ 0000000180006380     librawmonitor.obj
 0002:000013e8       ??_C@_0DN@NCPDJLOG@?$CIthreadName?5?$DN?5jni_env?9?$DONewStrin@ 00000001800063e8     librawmonitor.obj
 0002:00001430       ??_C@_0FE@PFKODBGC@?$CIthreadObject?5?$DN?5jni_env?9?$DONewObj@ 0000000180006430     librawmonitor.obj
 0002:00001490       ??_C@_0ED@HOBAHHJI@?$CIthreadGlobalRef?5?$DN?5jni_env?9?$DONew@ 0000000180006490     librawmonitor.obj
 0002:000014e0       ??_C@_0FN@HNJJAHFC@jvmti_env?9?$DORunAgentThread?$CIagent@ 00000001800064e0     librawmonitor.obj
 0002:00001540       ??_C@_0EA@MOJDNKDF@Debuggee?5status?5sync?5aborted?5be@ 0000000180006540     librawmonitor.obj
 0002:00001580       ??_C@_0EA@EEOEJAEN@status?5?$DN?5syncDebuggeeStatus?$CIjni@ 0000000180006580     librawmonitor.obj
 0002:000015c0       ??_C@_0BL@JBCFNBMB@nsk_jvmti_resetAgentData?$CI?$CJ@ 00000001800065c0     librawmonitor.obj
 0002:000015e0       ??_C@_0EL@LPBEELIP@s?2test?2hotspot?2jtreg?2vmTestbase@ 00000001800065e0     librawmonitor.obj
 0002:00001630       ??_C@_0CK@JDAMFDMJ@jvmti?9?$DOSetTag?$CIo?0?5tag?$CJ?5?$DN?$DN?5JVMTI_@ 0000000180006630     librawmonitor.obj
 0002:00001660       ??_C@_0CC@DAMNHKNI@Can?8t?5set?5tag?5?$CFli?5for?5object?5?$CFl@ 0000000180006660     librawmonitor.obj
 0002:00001688       ??_C@_0DL@HAJPNKEF@jvmti?9?$DOGetObjectHashCode?$CIo?0?5?$CGha@ 0000000180006688     librawmonitor.obj
 0002:000016c8       ??_C@_0BL@JFPIEOBF@Can?8t?5get?5hash?5object?5?$CFlx?6@ 00000001800066c8     librawmonitor.obj
 0002:000016e8       ??_C@_0BG@DICPHBKN@setTag?3?5?$CF08x?5?$DM?9?5?$CF?53li@ 00000001800066e8     librawmonitor.obj
 0002:00001700       ??_C@_0DH@FCEEBDMJ@?$CIs?5?$DN?5jni?9?$DOGetStringUTFChars?$CIsIn@ 0000000180006700     librawmonitor.obj
 0002:00001738       ??_C@_0BJ@OKKGHDCN@Can?8t?5get?5string?5at?5?$CF?$CDp?6@ 0000000180006738     librawmonitor.obj
 0002:00001758       ??_C@_0BP@EKFLGGFJ@Can?8t?5get?5string?5at?5?$CF?$CDp?3?5null?6@ 0000000180006758     librawmonitor.obj
 0002:00001778       ??_C@_06ICODBHCL@?5?1?1?5?$CFs@ 0000000180006778     librawmonitor.obj
 0002:00001780       ??_C@_0DB@KGFPLEGO@?$CIr?5?$DN?5jvmti?9?$DOGetTag?$CIo?0?5?$CGtag?$CJ?$CJ?5?$DN?$DN@ 0000000180006780     librawmonitor.obj
 0002:000017b8       ??_C@_0CO@PDAGBCGJ@Can?8t?5GetTag?5for?5object?5?$CFlx?4?5Re@ 00000001800067b8     librawmonitor.obj
 0002:000017e8       ??_C@_0CH@HPEODOHC@TEST_BUG?3?5Max?4?5number?5of?5refs?5r@ 00000001800067e8     librawmonitor.obj
 0002:00001810       ??_C@_0DI@PHFCABIM@?$CIr?5?$DN?5jvmti?9?$DOGetTag?$CIfrom?0?5?$CGtagFr@ 0000000180006810     librawmonitor.obj
 0002:00001848       ??_C@_0DI@MDEGFNKD@TEST_BUG?3?5Can?8t?5GetTag?5for?5obje@ 0000000180006848     librawmonitor.obj
 0002:00001880       ??_C@_0DE@MLELJAHM@?$CIr?5?$DN?5jvmti?9?$DOGetTag?$CIto?0?5?$CGtagTo?$CJ?$CJ@ 0000000180006880     librawmonitor.obj
 0002:000018b8       ??_C@_0CH@NDICEDBM@?5JVMTI?5GetCurrentThread?5returne@ 00000001800068b8     librawmonitor.obj
 0002:000018e0       ??_C@_04NKMBPDJM@?5?$CFd?6@ 00000001800068e0     librawmonitor.obj
 0002:000018e8       ??_C@_0BE@EEKKELIK@VMInit?5event?5?5done?6@ 00000001800068e8     librawmonitor.obj
 0002:00001900       ??_C@_0CB@OKPJJILN@?5Raw?5monitor?5exit?5returned?5erro@ 0000000180006900     librawmonitor.obj
 0002:00001928       ??_C@_0DA@JDIEHOA@?9?9?9?9?9?9?9?9?9?9?9?9?5JVMTI_EVENT_VM_DEA@ 0000000180006928     librawmonitor.obj
 0002:00001958       ??_C@_0BP@GKIKEIDG@?5JVMTI?5GetPhase?5returned?5error@ 0000000180006958     librawmonitor.obj
 0002:00001978       ??_C@_0DC@HNGPGPEK@?9?9?9?9?9?9?9?9?9?9?9?9?5classFileLoadHookE@ 0000000180006978     librawmonitor.obj
 0002:000019b0       ??_C@_0CA@OBGIPGLI@Raw?5monitor?5exit?5returned?5error@ 00000001800069b0     librawmonitor.obj
 0002:000019d0       ??_C@_0BG@CBLKFCHN@?5unexpected?5error?5?$CFd?6@ 00000001800069d0     librawmonitor.obj
 0002:000019e8       ??_C@_0CB@FNOAGBDP@Raw?5monitor?5enter?5returned?5erro@ 00000001800069e8     librawmonitor.obj
 0002:00001a10       ??_C@_09OPJEJKBL@printdump@ 0000000180006a10     librawmonitor.obj
 0002:00001a20       ??_C@_0CJ@KCDEKOCJ@Wrong?5result?5of?5a?5valid?5call?5to@ 0000000180006a20     librawmonitor.obj
 0002:00001a50       ??_C@_0N@HJAMKMBE@_access_lock@ 0000000180006a50     librawmonitor.obj
 0002:00001a60       ??_C@_0CJ@ONFKMPMM@CreateRawMonitor?5failed?5with?5er@ 0000000180006a60     librawmonitor.obj
 0002:00001a90       ??_C@_0BJ@MAOBBOBH@_access_lock_not_entered@ 0000000180006a90     librawmonitor.obj
 0002:00001ab0       ??_C@_0N@GLFGABJG@RawMonitor?90@ 0000000180006ab0     librawmonitor.obj
 0002:00001ac0       ??_C@_0CI@EDEMEGFA@GetPotentialCapabilities?5return@ 0000000180006ac0     librawmonitor.obj
 0002:00001ae8       ??_C@_0CB@NJBLABLF@SetEventCallbacks?5returned?5erro@ 0000000180006ae8     librawmonitor.obj
 0002:00001b10       ??_C@_0DE@MEFKDHFM@SetEventNotificationMode?5for?5VM@ 0000000180006b10     librawmonitor.obj
 0002:00001b48       ??_C@_0DL@KHAEEJDH@SetEventNotificationMode?5for?5vm@ 0000000180006b48     librawmonitor.obj
 0002:00001b88       ??_C@_0DN@PLAPDNNM@SetEventNotificationMode?5CLASS_@ 0000000180006b88     librawmonitor.obj
 0002:00001bc8       ??_C@_0CD@NHAPPFHC@Destroy?5Raw?5monitor?5returned?5er@ 0000000180006bc8     librawmonitor.obj
 0002:00001bf0       ??_C@_0O@IEOHCAJP@Rawmonitor?9?$CFd@ 0000000180006bf0     librawmonitor.obj
 0002:00001c00       ??_C@_0BL@PPNDBPKK@jvmti?5create?5raw?5monitor?5?6@ 0000000180006c00     librawmonitor.obj
 0002:00001c20       ??_C@_0BN@DELNHPGN@Error?3?5CreateRawMonitor?5?$CFd?5?6@ 0000000180006c20     librawmonitor.obj
 0002:00001c40       ??_C@_0BK@KEFLCGDC@jvmti?5Raw?5monitor?5enter?5?6@ 0000000180006c40     librawmonitor.obj
 0002:00001c60       ??_C@_0BM@DDMCJCDD@Error?3?5RawMonitorEnter?5?$CFd?5?6@ 0000000180006c60     librawmonitor.obj
 0002:00001c80       ??_C@_0BJ@OJLKHENF@jvmti?5raw?5monitor?5exit?5?6@ 0000000180006c80     librawmonitor.obj
 0002:00001ca0       ??_C@_0BL@GKGBEHOI@Error?3?5RawMonitorExit?5?$CFd?5?6@ 0000000180006ca0     librawmonitor.obj
 0002:00001cc0       ??_C@_0BH@PILJFGHG@jvmti?5RawMonitorWait?5?6@ 0000000180006cc0     librawmonitor.obj
 0002:00001cd8       ??_C@_0BL@EJFJOCBH@Error?3?5RawMonitorWait?5?$CFd?5?6@ 0000000180006cd8     librawmonitor.obj
 0002:00001d10       ??_C@_1EC@JIJBPKFM@?$AAa?$AAp?$AAi?$AA?9?$AAm?$AAs?$AA?9?$AAw?$AAi?$AAn?$AA?9?$AAc?$AAo?$AAr?$AAe@ 0000000180006d10     MSVCRT:thread_safe_statics.obj
 0002:00001d58       ??_C@_1BK@MGMFAEKH@?$AAk?$AAe?$AAr?$AAn?$AAe?$AAl?$AA3?$AA2?$AA?4?$AAd?$AAl?$AAl@ 0000000180006d58     MSVCRT:thread_safe_statics.obj
 0002:00001d78       ??_C@_0BJ@JEBJOJFJ@SleepConditionVariableCS@ 0000000180006d78     MSVCRT:thread_safe_statics.obj
 0002:00001d98       ??_C@_0BJ@PGPPEPCC@WakeAllConditionVariable@ 0000000180006d98     MSVCRT:thread_safe_statics.obj
 0002:00001db8       _pDefaultRawDllMain        0000000180006db8     MSVCRT:dll_dllmain.obj
 0002:00001db8       _pRawDllMain               0000000180006db8     MSVCRT:dll_dllmain.obj
 0002:00001dc0       __xmm@ffffffffffffffffffffffffffffffff 0000000180006dc0     MSVCRT:utility.obj
 0002:00001dd0       _load_config_used          0000000180006dd0     MSVCRT:loadcfg.obj
 0002:00001f80       _tls_used                  0000000180006f80     MSVCRT:tlssup.obj
 0002:00001fa8       __volatile_metadata        0000000180006fa8     <linker-defined>
 0002:00002378       __rtc_iaa                  0000000180007378     MSVCRT:initsect.obj
 0002:00002380       __rtc_izz                  0000000180007380     MSVCRT:initsect.obj
 0002:00002388       __rtc_taa                  0000000180007388     MSVCRT:initsect.obj
 0002:00002390       __rtc_tzz                  0000000180007390     MSVCRT:initsect.obj
 0002:00002398       _tls_start                 0000000180007398     MSVCRT:tlssup.obj
 0002:0000239c       _Init_thread_epoch         000000018000739c     MSVCRT:thread_safe_statics.obj
 0002:000023a0       _tls_end                   00000001800073a0     MSVCRT:tlssup.obj
 0002:00002b5c       __IMPORT_DESCRIPTOR_KERNEL32 0000000180007b5c     kernel32:KERNEL32.dll
 0002:00002b70       __IMPORT_DESCRIPTOR_VCRUNTIME140 0000000180007b70     vcruntime:VCRUNTIME140.dll
 0002:00002b84       __IMPORT_DESCRIPTOR_api-ms-win-crt-runtime-l1-1-0 0000000180007b84     ucrt:api-ms-win-crt-runtime-l1-1-0.dll
 0002:00002b98       __IMPORT_DESCRIPTOR_api-ms-win-crt-stdio-l1-1-0 0000000180007b98     ucrt:api-ms-win-crt-stdio-l1-1-0.dll
 0002:00002bac       __IMPORT_DESCRIPTOR_api-ms-win-crt-string-l1-1-0 0000000180007bac     ucrt:api-ms-win-crt-string-l1-1-0.dll
 0002:00002bc0       __NULL_IMPORT_DESCRIPTOR   0000000180007bc0     kernel32:KERNEL32.dll
 0003:00000034       _Init_global_epoch         0000000180009034     MSVCRT:thread_safe_statics.obj
 0003:00000040       __security_cookie          0000000180009040     MSVCRT:gs_cookie.obj
 0003:00000048       __security_cookie_complement 0000000180009048     MSVCRT:gs_cookie.obj
 0003:00000050       __scrt_native_dllmain_reason 0000000180009050     MSVCRT:utility.obj
 0003:00000058       __isa_available            0000000180009058     MSVCRT:cpu_disp.obj
 0003:0000005c       __isa_enabled              000000018000905c     MSVCRT:cpu_disp.obj
 0003:00000060       __memset_fast_string_threshold 0000000180009060     MSVCRT:cpu_disp.obj
 0003:00000068       __memset_nt_threshold      0000000180009068     MSVCRT:cpu_disp.obj
 0003:00000070       __scrt_ucrt_dll_is_in_use  0000000180009070     MSVCRT:ucrt_stubs.obj
 0003:00000080       g_wrongHeapCallbacks       0000000180009080     librawmonitor.obj
 0003:00000100       g_szTagInfo                0000000180009100     librawmonitor.obj
 0003:00002040       g_tagFlags                 000000018000b040     librawmonitor.obj
 0003:00002428       g_refsToVerifyCnt          000000018000b428     librawmonitor.obj
 0003:0000242c       g_fakeUserData             000000018000b42c     librawmonitor.obj
 0003:00002430       g_tagVisitCount            000000018000b430     librawmonitor.obj
 0003:000033d0       g_refsToVerify             000000018000c3d0     librawmonitor.obj
 0003:0001aad0       g_userDataError            0000000180023ad0     librawmonitor.obj
 0003:0001aad4       iGlobalStatus              0000000180023ad4     librawmonitor.obj
 0003:0001aad8       access_lock                0000000180023ad8     librawmonitor.obj
 0003:0001aae0       access_lock_not_entered    0000000180023ae0     librawmonitor.obj
 0003:0001aae8       jvmti                      0000000180023ae8     librawmonitor.obj
 0003:0001aaf0       main_thread                0000000180023af0     librawmonitor.obj
 0003:0001aaf8       printdump                  0000000180023af8     librawmonitor.obj
 0003:0001ab00       jraw_monitor               0000000180023b00     librawmonitor.obj
 0003:0001ae78       ?_OptionsStorage@?1??__local_stdio_printf_options@@9@4_KA 0000000180023e78     librawmonitor.obj
 0003:0001b438       _tls_index                 0000000180024438     MSVCRT:tlssup.obj
 0003:0001b440       __scrt_current_native_startup_state 0000000180024440     MSVCRT:utility.obj
 0003:0001b448       __scrt_native_startup_lock 0000000180024448     MSVCRT:utility.obj
 0003:0001b488       __scrt_debugger_hook_flag  0000000180024488     MSVCRT:utility_desktop.obj
 0003:0001b490       ?__type_info_root_node@@3U__type_info_node@@A 0000000180024490     MSVCRT:tncleanup.obj
 0003:0001b4a0       ?_OptionsStorage@?1??__local_stdio_scanf_options@@9@4_KA 00000001800244a0     MSVCRT:default_local_stdio_options.obj
 0003:0001b4a8       __favor                    00000001800244a8     MSVCRT:cpu_disp.obj
 0003:0001b4b0       __dyn_tls_init_callback    00000001800244b0     <common>

 entry point at        0001:00002950

 Static symbols

 0000:fffd9000       .debug$S                   0000000180000000     rawmonitor.exp
 0000:fffd9000       .debug$S                   0000000180000000     vcruntime:VCRUNTIME140.dll
 0000:fffd9000       .debug$S                   0000000180000000     vcruntime:VCRUNTIME140.dll
 0000:fffd9000       .debug$S                   0000000180000000     vcruntime:VCRUNTIME140.dll
 0000:fffd9000       .debug$S                   0000000180000000     vcruntime:VCRUNTIME140.dll
 0000:fffd9000       .debug$S                   0000000180000000     vcruntime:VCRUNTIME140.dll
 0000:fffd9000       .debug$S                   0000000180000000     vcruntime:VCRUNTIME140.dll
 0000:fffd9000       .debug$S                   0000000180000000     vcruntime:VCRUNTIME140.dll
 0000:fffd9000       .debug$S                   0000000180000000     vcruntime:VCRUNTIME140.dll
 0000:fffd9000       .debug$S                   0000000180000000     ucrt:api-ms-win-crt-convert-l1-1-0.dll
 0002:ffffb000       .idata$6                   0000000180000000     ucrt:api-ms-win-crt-convert-l1-1-0.dll
 0000:fffd9000       .debug$S                   0000000180000000     ucrt:api-ms-win-crt-heap-l1-1-0.dll
 0000:fffd9000       .debug$S                   0000000180000000     ucrt:api-ms-win-crt-heap-l1-1-0.dll
 0000:fffd9000       .debug$S                   0000000180000000     ucrt:api-ms-win-crt-heap-l1-1-0.dll
 0000:fffd9000       .debug$S                   0000000180000000     ucrt:api-ms-win-crt-heap-l1-1-0.dll
 0002:ffffb000       .idata$6                   0000000180000000     ucrt:api-ms-win-crt-heap-l1-1-0.dll
 0000:fffd9000       .debug$S                   0000000180000000     ucrt:api-ms-win-crt-runtime-l1-1-0.dll
 0000:fffd9000       .debug$S                   0000000180000000     ucrt:api-ms-win-crt-runtime-l1-1-0.dll
 0000:fffd9000       .debug$S                   0000000180000000     ucrt:api-ms-win-crt-runtime-l1-1-0.dll
 0000:fffd9000       .debug$S                   0000000180000000     ucrt:api-ms-win-crt-runtime-l1-1-0.dll
 0000:fffd9000       .debug$S                   0000000180000000     ucrt:api-ms-win-crt-runtime-l1-1-0.dll
 0000:fffd9000       .debug$S                   0000000180000000     ucrt:api-ms-win-crt-runtime-l1-1-0.dll
 0000:fffd9000       .debug$S                   0000000180000000     ucrt:api-ms-win-crt-runtime-l1-1-0.dll
 0000:fffd9000       .debug$S                   0000000180000000     ucrt:api-ms-win-crt-runtime-l1-1-0.dll
 0000:fffd9000       .debug$S                   0000000180000000     ucrt:api-ms-win-crt-runtime-l1-1-0.dll
 0000:fffd9000       .debug$S                   0000000180000000     ucrt:api-ms-win-crt-runtime-l1-1-0.dll
 0000:fffd9000       .debug$S                   0000000180000000     ucrt:api-ms-win-crt-runtime-l1-1-0.dll
 0000:fffd9000       .debug$S                   0000000180000000     ucrt:api-ms-win-crt-runtime-l1-1-0.dll
 0000:fffd9000       .debug$S                   0000000180000000     ucrt:api-ms-win-crt-runtime-l1-1-0.dll
 0000:fffd9000       .debug$S                   0000000180000000     ucrt:api-ms-win-crt-runtime-l1-1-0.dll
 0000:fffd9000       .debug$S                   0000000180000000     ucrt:api-ms-win-crt-runtime-l1-1-0.dll
 0000:fffd9000       .debug$S                   0000000180000000     ucrt:api-ms-win-crt-runtime-l1-1-0.dll
 0000:fffd9000       .debug$S                   0000000180000000     ucrt:api-ms-win-crt-stdio-l1-1-0.dll
 0000:fffd9000       .debug$S                   0000000180000000     ucrt:api-ms-win-crt-stdio-l1-1-0.dll
 0000:fffd9000       .debug$S                   0000000180000000     ucrt:api-ms-win-crt-stdio-l1-1-0.dll
 0000:fffd9000       .debug$S                   0000000180000000     ucrt:api-ms-win-crt-stdio-l1-1-0.dll
 0000:fffd9000       .debug$S                   0000000180000000     ucrt:api-ms-win-crt-stdio-l1-1-0.dll
 0000:fffd9000       .debug$S                   0000000180000000     ucrt:api-ms-win-crt-stdio-l1-1-0.dll
 0000:fffd9000       .debug$S                   0000000180000000     ucrt:api-ms-win-crt-stdio-l1-1-0.dll
 0000:fffd9000       .debug$S                   0000000180000000     ucrt:api-ms-win-crt-stdio-l1-1-0.dll
 0000:fffd9000       .debug$S                   0000000180000000     ucrt:api-ms-win-crt-stdio-l1-1-0.dll
 0000:fffd9000       .debug$S                   0000000180000000     ucrt:api-ms-win-crt-stdio-l1-1-0.dll
 0000:fffd9000       .debug$S                   0000000180000000     ucrt:api-ms-win-crt-string-l1-1-0.dll
 0000:fffd9000       .debug$S                   0000000180000000     ucrt:api-ms-win-crt-string-l1-1-0.dll
 0000:fffd9000       .debug$S                   0000000180000000     ucrt:api-ms-win-crt-string-l1-1-0.dll
 0000:fffd9000       .debug$S                   0000000180000000     ucrt:api-ms-win-crt-string-l1-1-0.dll
 0000:fffd9000       .debug$S                   0000000180000000     ucrt:api-ms-win-crt-string-l1-1-0.dll
 0000:fffd9000       .debug$S                   0000000180000000     ucrt:api-ms-win-crt-string-l1-1-0.dll
 0000:fffd9000       .debug$S                   0000000180000000     ucrt:api-ms-win-crt-string-l1-1-0.dll
 0000:fffd9000       .debug$S                   0000000180000000     ucrt:api-ms-win-crt-string-l1-1-0.dll
 0000:fffd9000       .debug$S                   0000000180000000     kernel32:KERNEL32.dll
 0000:fffd9000       .debug$S                   0000000180000000     kernel32:KERNEL32.dll
 0000:fffd9000       .debug$S                   0000000180000000     kernel32:KERNEL32.dll
 0000:fffd9000       .debug$S                   0000000180000000     kernel32:KERNEL32.dll
 0000:fffd9000       .debug$S                   0000000180000000     kernel32:KERNEL32.dll
 0000:fffd9000       .debug$S                   0000000180000000     kernel32:KERNEL32.dll
 0000:fffd9000       .debug$S                   0000000180000000     kernel32:KERNEL32.dll
 0000:fffd9000       .debug$S                   0000000180000000     kernel32:KERNEL32.dll
 0000:fffd9000       .debug$S                   0000000180000000     kernel32:KERNEL32.dll
 0000:fffd9000       .debug$S                   0000000180000000     kernel32:KERNEL32.dll
 0000:fffd9000       .debug$S                   0000000180000000     kernel32:KERNEL32.dll
 0000:fffd9000       .debug$S                   0000000180000000     kernel32:KERNEL32.dll
 0000:fffd9000       .debug$S                   0000000180000000     kernel32:KERNEL32.dll
 0000:fffd9000       .debug$S                   0000000180000000     kernel32:KERNEL32.dll
 0000:fffd9000       .debug$S                   0000000180000000     kernel32:KERNEL32.dll
 0000:fffd9000       .debug$S                   0000000180000000     kernel32:KERNEL32.dll
 0000:fffd9000       .debug$S                   0000000180000000     kernel32:KERNEL32.dll
 0000:fffd9000       .debug$S                   0000000180000000     kernel32:KERNEL32.dll
 0000:fffd9000       .debug$S                   0000000180000000     kernel32:KERNEL32.dll
 0000:fffd9000       .debug$S                   0000000180000000     kernel32:KERNEL32.dll
 0000:fffd9000       .debug$S                   0000000180000000     kernel32:KERNEL32.dll
 0000:fffd9000       .debug$S                   0000000180000000     kernel32:KERNEL32.dll
 0000:fffd9000       .debug$S                   0000000180000000     kernel32:KERNEL32.dll
 0000:fffd9000       .debug$S                   0000000180000000     kernel32:KERNEL32.dll
 0000:fffd9000       .debug$S                   0000000180000000     kernel32:KERNEL32.dll
 0000:fffd9000       .debug$S                   0000000180000000     kernel32:KERNEL32.dll
 0000:fffd9000       .debug$S                   0000000180000000     kernel32:KERNEL32.dll
 0000:fffd9000       .debug$S                   0000000180000000     kernel32:KERNEL32.dll
 0001:00001228       addRefToVerify             0000000180002228 f   librawmonitor.obj
 0001:0000129c       agentThreadWrapper         000000018000229c f   librawmonitor.obj
 0001:000016c4       file_basename              00000001800026c4 f   librawmonitor.obj
 0001:00001d44       startAgentThreadWrapper    0000000180002d44 f   librawmonitor.obj
 0001:00002070       syncDebuggeeStatus         0000000180003070 f   librawmonitor.obj
 0001:00002410       capture_previous_context   0000000180003410 f   MSVCRT:gs_report.obj
 0001:00002484       ?__scrt_initialize_thread_safe_statics@@YAHXZ 0000000180003484 f   MSVCRT:thread_safe_statics.obj
 0001:00002554       ?__scrt_uninitialize_thread_safe_statics@@YAXXZ 0000000180003554 f   MSVCRT:thread_safe_statics.obj
 0001:00002600       $$000000                   0000000180003600     MSVCRT:amdsecgs.obj
 0001:00002630       ?dllmain_crt_dispatch@@YAHQEAUHINSTANCE__@@KQEAX@Z 0000000180003630 f   MSVCRT:dll_dllmain.obj
 0001:00002680       ?dllmain_crt_process_attach@@YAHQEAUHINSTANCE__@@QEAX@Z 0000000180003680 f   MSVCRT:dll_dllmain.obj
 0001:00002798       ?dllmain_crt_process_detach@@YAH_N@Z 0000000180003798 f   MSVCRT:dll_dllmain.obj
 0001:0000281c       ?dllmain_dispatch@@YAHQEAUHINSTANCE__@@KQEAX@Z 000000018000381c f   MSVCRT:dll_dllmain.obj
 0001:00003230       $$000000                   0000000180004230     MSVCRT:guard_dispatch.obj
 0001:00003250       $$000000                   0000000180004250     MSVCRT:guard_xfg_dispatch.obj
 0001:00003266       ?fin$0@?0??dllmain_crt_process_attach@@YAHQEAUHINSTANCE__@@QEAX@Z@4HA 0000000180004266 f   MSVCRT:dll_dllmain.obj
 0001:0000327d       ?fin$0@?0??dllmain_crt_process_detach@@YAH_N@Z@4HA 000000018000427d f   MSVCRT:dll_dllmain.obj
 0001:00003296       ?fin$1@?0??dllmain_crt_process_detach@@YAH_N@Z@4HA 0000000180004296 f   MSVCRT:dll_dllmain.obj
 0001:000032aa       ?filt$0@?0??dllmain_dispatch@@YAHQEAUHINSTANCE__@@KQEAX@Z@4HA 00000001800042aa f   MSVCRT:dll_dllmain.obj
 0001:000032e0       __scrt_is_nonwritable_in_current_image$filt$0 00000001800042e0 f   MSVCRT:utility.obj
 0002:000001e8       ?__scrt_initialize_tss_var@@3P6AHXZEA 00000001800051e8     MSVCRT:thread_safe_statics.obj
 0002:00000310       ?opcLengths@@3QBEB         0000000180005310     librawmonitor.obj
 0002:00001cf8       GS_ExceptionPointers       0000000180006cf8     MSVCRT:gs_report.obj
 0002:000023a8       $unwind$fprintf            00000001800073a8     librawmonitor.obj
 0002:000023b4       $unwind$debug_printf       00000001800073b4     librawmonitor.obj
 0002:000023b4       $unwind$printf             00000001800073b4     librawmonitor.obj
 0002:000023c0       $unwind$_snprintf          00000001800073c0     librawmonitor.obj
 0002:000023d0       $unwind$?NewObject@JNIEnv_@@QEAAPEAV_jobject@@PEAV_jclass@@PEAU_jmethodID@@ZZ 00000001800073d0     librawmonitor.obj
 0002:000023d0       $unwind$nsk_lcomplain      00000001800073d0     librawmonitor.obj
 0002:000023d0       $unwind$nsk_ldisplay       00000001800073d0     librawmonitor.obj
 0002:000023d8       $unwind$nsk_lvdisplay      00000001800073d8     librawmonitor.obj
 0002:000023d8       $unwind$vmInit             00000001800073d8     librawmonitor.obj
 0002:000023d8       $unwind$vmStart            00000001800073d8     librawmonitor.obj
 0002:000023d8       $unwind$_RTC_Initialize    00000001800073d8     MSVCRT:initsect.obj
 0002:000023d8       $unwind$_RTC_Terminate     00000001800073d8     MSVCRT:initsect.obj
 0002:000023d8       $unwind$?__scrt_initialize_thread_safe_statics@@YAHXZ 00000001800073d8     MSVCRT:thread_safe_statics.obj
 0002:000023e4       $unwind$nsk_lvcomplain     00000001800073e4     librawmonitor.obj
 0002:000023fc       $unwind$nsk_ltrace         00000001800073fc     librawmonitor.obj
 0002:000023fc       $unwind$__report_gsfailure 00000001800073fc     MSVCRT:gs_report.obj
 0002:00002404       $unwind$Java_nsk_jvmti_unit_functions_rawmonitor_RawMonitorEnter 0000000180007404     librawmonitor.obj
 0002:00002404       $unwind$Java_nsk_jvmti_unit_functions_rawmonitor_RawMonitorExit 0000000180007404     librawmonitor.obj
 0002:00002404       $unwind$Java_nsk_jvmti_unit_functions_rawmonitor_RawMonitorWait 0000000180007404     librawmonitor.obj
 0002:00002404       $unwind$nsk_lvtrace        0000000180007404     librawmonitor.obj
 0002:00002404       $unwind$__raise_securityfailure 0000000180007404     MSVCRT:gs_report.obj
 0002:00002404       $unwind$__scrt_initialize_crt 0000000180007404     MSVCRT:utility.obj
 0002:00002404       $unwind$__scrt_initialize_onexit_tables 0000000180007404     MSVCRT:utility.obj
 0002:00002404       $unwind$__scrt_release_startup_lock 0000000180007404     MSVCRT:utility.obj
 0002:00002404       $unwind$__scrt_uninitialize_crt 0000000180007404     MSVCRT:utility.obj
 0002:00002404       $unwind$_onexit            0000000180007404     MSVCRT:utility.obj
 0002:0000240c       $unwind$nsk_lverify        000000018000740c     librawmonitor.obj
 0002:0000241c       $unwind$nsk_vprintf        000000018000741c     librawmonitor.obj
 0002:0000242c       $unwind$nsk_printf         000000018000742c     librawmonitor.obj
 0002:00002434       $unwind$?nsk_jni_lverify@@YAHHPEAUJNIEnv_@@HQEBDH1ZZ 0000000180007434     librawmonitor.obj
 0002:00002448       $unwind$?nsk_jni_check_exception@@YAHPEAUJNIEnv_@@QEBDH@Z 0000000180007448     librawmonitor.obj
 0002:00002464       $unwind$Java_nsk_jvmti_unit_FollowReferences_FollowRefObjects_resetTags 0000000180007464     librawmonitor.obj
 0002:00002464       $unwind$addRefToVerify     0000000180007464     librawmonitor.obj
 0002:00002464       $unwind$init_callbacks     0000000180007464     librawmonitor.obj
 0002:00002464       $unwind$nsk_jvmti_resetAgentData 0000000180007464     librawmonitor.obj
 0002:00002464       $unwind$__scrt_initialize_default_local_stdio_options 0000000180007464     MSVCRT:default_local_stdio_options.obj
 0002:00002464       $unwind$?dllmain_crt_dispatch@@YAHQEAUHINSTANCE__@@KQEAX@Z 0000000180007464     MSVCRT:dll_dllmain.obj
 0002:00002464       $unwind$DllMain            0000000180007464     MSVCRT:dll_dllmain_stub.obj
 0002:00002464       $unwind$__GSHandlerCheck   0000000180007464     MSVCRT:gshandler.obj
 0002:00002464       $unwind$?__scrt_uninitialize_thread_safe_statics@@YAXXZ 0000000180007464     MSVCRT:thread_safe_statics.obj
 0002:00002464       $unwind$__scrt_acquire_startup_lock 0000000180007464     MSVCRT:utility.obj
 0002:00002464       $unwind$__scrt_dllmain_after_initialize_c 0000000180007464     MSVCRT:utility.obj
 0002:00002464       $unwind$__scrt_dllmain_before_initialize_c 0000000180007464     MSVCRT:utility.obj
 0002:00002464       $unwind$__scrt_dllmain_crt_thread_attach 0000000180007464     MSVCRT:utility.obj
 0002:00002464       $unwind$__scrt_dllmain_crt_thread_detach 0000000180007464     MSVCRT:utility.obj
 0002:00002464       $unwind$__scrt_dllmain_uninitialize_c 0000000180007464     MSVCRT:utility.obj
 0002:00002464       $unwind$__scrt_dllmain_uninitialize_critical 0000000180007464     MSVCRT:utility.obj
 0002:00002464       $unwind$atexit             0000000180007464     MSVCRT:utility.obj
 0002:0000246c       $unwind$nsk_jvmti_lverify  000000018000746c     librawmonitor.obj
 0002:00002480       $unwind$exitOnError        0000000180007480     librawmonitor.obj
 0002:00002490       $unwind$Java_nsk_share_jvmti_ArgumentHandler_getAgentOptionsString 0000000180007490     librawmonitor.obj
 0002:000024a4       $unwind$Java_nsk_jvmti_unit_FollowReferences_FollowRefObjects_getTag 00000001800074a4     librawmonitor.obj
 0002:000024a4       $unwind$Java_nsk_share_jvmti_DebugeeClass_checkStatus 00000001800074a4     librawmonitor.obj
 0002:000024a4       $unwind$agentThreadWrapper 00000001800074a4     librawmonitor.obj
 0002:000024b4       $unwind$startAgentThreadWrapper 00000001800074b4     librawmonitor.obj
 0002:000024d0       $unwind$syncDebuggeeStatus 00000001800074d0     librawmonitor.obj
 0002:000024d0       $unwind$__scrt_dllmain_exception_filter 00000001800074d0     MSVCRT:utility.obj
 0002:000024e4       $unwind$Java_nsk_share_jvmti_DebugeeClass_resetAgentData 00000001800074e4     librawmonitor.obj
 0002:000024ec       $unwind$MA_checkStatus     00000001800074ec     librawmonitor.obj
 0002:00002500       $unwind$Java_nsk_jvmti_unit_FollowReferences_FollowRefObjects_setTag 0000000180007500     librawmonitor.obj
 0002:00002518       $unwind$Java_nsk_jvmti_unit_FollowReferences_FollowRefObjects_addRefToVerify 0000000180007518     librawmonitor.obj
 0002:00002534       $unwind$Agent_Initialize   0000000180007534     librawmonitor.obj
 0002:00002534       $unwind$_DllMainCRTStartup 0000000180007534     MSVCRT:dll_dllmain.obj
 0002:00002544       $unwind$classFileLoadHookEvent 0000000180007544     librawmonitor.obj
 0002:00002558       $unwind$Java_nsk_jvmti_unit_functions_rawmonitor_CreateRawMonitor 0000000180007558     librawmonitor.obj
 0002:0000256c       $unwind$capture_previous_context 000000018000756c     MSVCRT:gs_report.obj
 0002:00002578       $unwind$__GSHandlerCheckCommon 0000000180007578     MSVCRT:gshandler.obj
 0002:00002580       $xdatasym                  0000000180007580     MSVCRT:amdsecgs.obj
 0002:00002584       $unwind$?dllmain_crt_process_attach@@YAHQEAUHINSTANCE__@@QEAX@Z 0000000180007584     MSVCRT:dll_dllmain.obj
 0002:000025c0       $unwind$?fin$0@?0??dllmain_crt_process_attach@@YAHQEAUHINSTANCE__@@QEAX@Z@4HA 00000001800075c0     MSVCRT:dll_dllmain.obj
 0002:000025c0       $unwind$?fin$0@?0??dllmain_crt_process_detach@@YAH_N@Z@4HA 00000001800075c0     MSVCRT:dll_dllmain.obj
 0002:000025c0       $unwind$?fin$1@?0??dllmain_crt_process_detach@@YAH_N@Z@4HA 00000001800075c0     MSVCRT:dll_dllmain.obj
 0002:000025c8       $unwind$?dllmain_crt_process_detach@@YAH_N@Z 00000001800075c8     MSVCRT:dll_dllmain.obj
 0002:0000261c       $unwind$?dllmain_dispatch@@YAHQEAUHINSTANCE__@@KQEAX@Z 000000018000761c     MSVCRT:dll_dllmain.obj
 0002:00002644       $unwind$?filt$0@?0??dllmain_dispatch@@YAHQEAUHINSTANCE__@@KQEAX@Z@4HA 0000000180007644     MSVCRT:dll_dllmain.obj
 0002:0000264c       $unwind$__scrt_is_nonwritable_in_current_image 000000018000764c     MSVCRT:utility.obj
 0002:0000266c       $unwind$__scrt_is_nonwritable_in_current_image$filt$0 000000018000766c     MSVCRT:utility.obj
 0002:00002674       $unwind$__scrt_fastfail    0000000180007674     MSVCRT:utility_desktop.obj
 0002:00002684       $unwind$__security_init_cookie 0000000180007684     MSVCRT:gs_support.obj
 0002:00002690       $unwind$__isa_available_init 0000000180007690     MSVCRT:cpu_disp.obj
 0002:000026a0       $xdatasym                  00000001800076a0     MSVCRT:guard_dispatch.obj
 0002:000026a8       $xdatasym                  00000001800076a8     MSVCRT:guard_xfg_dispatch.obj
 0002:000026b0       .edata                     00000001800076b0     rawmonitor.exp
 0002:000026d8       rgpv                       00000001800076d8     rawmonitor.exp
 0002:00002724       rgszName                   0000000180007724     rawmonitor.exp
 0002:00002770       rgwOrd                     0000000180007770     rawmonitor.exp
 0002:00002796       szName                     0000000180007796     rawmonitor.exp
 0002:000027a5       $N00001                    00000001800077a5     rawmonitor.exp
 0002:000027b4       $N00002                    00000001800077b4     rawmonitor.exp
 0002:000027c1       $N00003                    00000001800077c1     rawmonitor.exp
 0002:00002806       $N00004                    0000000180007806     rawmonitor.exp
 0002:00002843       $N00005                    0000000180007843     rawmonitor.exp
 0002:0000288b       $N00006                    000000018000788b     rawmonitor.exp
 0002:000028cb       $N00007                    00000001800078cb     rawmonitor.exp
 0002:00002908       $N00008                    0000000180007908     rawmonitor.exp
 0002:00002942       $N00009                    0000000180007942     rawmonitor.exp
 0002:00002975       $N00010                    0000000180007975     rawmonitor.exp
 0002:000029ae       $N00011                    00000001800079ae     rawmonitor.exp
 0002:000029e6       $N00012                    00000001800079e6     rawmonitor.exp
 0002:00002a1e       $N00013                    0000000180007a1e     rawmonitor.exp
 0002:00002a59       $N00014                    0000000180007a59     rawmonitor.exp
 0002:00002a87       $N00015                    0000000180007a87     rawmonitor.exp
 0002:00002ab8       $N00016                    0000000180007ab8     rawmonitor.exp
 0002:00002ae7       $N00017                    0000000180007ae7     rawmonitor.exp
 0002:00002b16       $N00018                    0000000180007b16     rawmonitor.exp
 0002:00002b4b       $N00019                    0000000180007b4b     rawmonitor.exp
 0002:00002f5a       .idata$6                   0000000180007f5a     kernel32:KERNEL32.dll
 0002:00002fc8       .idata$6                   0000000180007fc8     vcruntime:VCRUNTIME140.dll
 0002:0000312a       .idata$6                   000000018000812a     ucrt:api-ms-win-crt-runtime-l1-1-0.dll
 0002:0000314c       .idata$6                   000000018000814c     ucrt:api-ms-win-crt-stdio-l1-1-0.dll
 0002:0000316c       .idata$6                   000000018000816c     ucrt:api-ms-win-crt-string-l1-1-0.dll
 0003:00000000       ?codeAttributeName@@3PEBDEB 0000000180009000     librawmonitor.obj
 0003:00000008       ?lineNumberAttributeName@@3PEBDEB 0000000180009008     librawmonitor.obj
 0003:00000010       ?localVarAttributeName@@3PEBDEB 0000000180009010     librawmonitor.obj
 0003:00000018       ?localVarTypeAttributeName@@3PEBDEB 0000000180009018     librawmonitor.obj
 0003:00000020       ?stackMapAttributeName@@3PEBDEB 0000000180009020     librawmonitor.obj
 0003:00000028       ?callBytes@@3PAEA          0000000180009028     librawmonitor.obj
 0003:0000002c       ?allocBytes@@3PAEA         000000018000902c     librawmonitor.obj
 0003:00000030       process_once               0000000180009030     librawmonitor.obj
 0003:0001aba0       nsk_context                0000000180023ba0     librawmonitor.obj
 0003:0001abac       redefineAttempted          0000000180023bac     librawmonitor.obj
 0003:0001abb0       redefineSucceed            0000000180023bb0     librawmonitor.obj
 0003:0001abb4       agentFailed                0000000180023bb4     librawmonitor.obj
 0003:0001abb8       agentThread                0000000180023bb8     librawmonitor.obj
 0003:0001abc0       context                    0000000180023bc0     librawmonitor.obj
 0003:0001ac78       agentThreadProc            0000000180023c78     librawmonitor.obj
 0003:0001ac80       agentThreadArg             0000000180023c80     librawmonitor.obj
 0003:0001ac88       agent_data                 0000000180023c88     librawmonitor.obj
 0003:0001ac98       jvmti_env                  0000000180023c98     librawmonitor.obj
 0003:0001aca0       jvm                        0000000180023ca0     librawmonitor.obj
 0003:0001aca8       jni_env                    0000000180023ca8     librawmonitor.obj
 0003:0001acb0       currentAgentStatus         0000000180023cb0     librawmonitor.obj
 0003:0001acb4       ?codeAttributeIndex@@3GA   0000000180023cb4     librawmonitor.obj
 0003:0001acb8       checkStatus_func           0000000180023cb8     librawmonitor.obj
 0003:0001acc0       ?lineNumberAttributeIndex@@3GA 0000000180023cc0     librawmonitor.obj
 0003:0001acc4       ?localVarAttributeIndex@@3GA 0000000180023cc4     librawmonitor.obj
 0003:0001acc8       ?localVarTypeAttributeIndex@@3GA 0000000180023cc8     librawmonitor.obj
 0003:0001accc       ?stackMapAttributeIndex@@3GA 0000000180023ccc     librawmonitor.obj
 0003:0001acd0       ?stackFrameOffset@@3GA     0000000180023cd0     librawmonitor.obj
 0003:0001acd4       ?mode@@3HA                 0000000180023cd4     librawmonitor.obj
 0003:0001acd8       ?orig@@3PEBEEB             0000000180023cd8     librawmonitor.obj
 0003:0001ace0       ?gen@@3PEAEEA              0000000180023ce0     librawmonitor.obj
 0003:0001ace8       ?inputPos@@3PEAEEA         0000000180023ce8     librawmonitor.obj
 0003:0001acf0       ?endPos@@3PEBEEB           0000000180023cf0     librawmonitor.obj
 0003:0001acf8       ?genPos@@3PEAEEA           0000000180023cf8     librawmonitor.obj
 0003:0001ad00       ?markPos@@3PEAEEA          0000000180023d00     librawmonitor.obj
 0003:0001ad08       ?constantPool@@3PEAPEADEA  0000000180023d08     librawmonitor.obj
 0003:0001ad10       ?constantPoolSize@@3GA     0000000180023d10     librawmonitor.obj
 0003:0001ad14       ?constantPoolCount@@3GA    0000000180023d14     librawmonitor.obj
 0003:0001ad18       ?zeroBytes@@3PAEA          0000000180023d18     librawmonitor.obj
 0003:0001ad1c       ?codeLength@@3IA           0000000180023d1c     librawmonitor.obj
 0003:0001ad20       ?map@@3PEAIEA              0000000180023d20     librawmonitor.obj
 0003:0001ad28       ?widening@@3PEACEA         0000000180023d28     librawmonitor.obj
 0003:0001ad30       callbacks                  0000000180023d30     librawmonitor.obj
 0003:0001ae68       jvmti_caps                 0000000180023e68     librawmonitor.obj
 0003:0001ae80       GS_ExceptionRecord         0000000180023e80     MSVCRT:gs_report.obj
 0003:0001af20       GS_ContextRecord           0000000180023f20     MSVCRT:gs_report.obj
 0003:0001b3f0       ?g_tss_cv@@3U_RTL_CONDITION_VARIABLE@@A 00000001800243f0     MSVCRT:thread_safe_statics.obj
 0003:0001b3f8       ?g_tss_event@@3PEAXEA      00000001800243f8     MSVCRT:thread_safe_statics.obj
 0003:0001b400       ?g_tss_mutex@@3U_RTL_CRITICAL_SECTION@@A 0000000180024400     MSVCRT:thread_safe_statics.obj
 0003:0001b428       ?g_sleep_condition_variable_cs@@3P6AHPEAU_RTL_CONDITION_VARIABLE@@PEAU_RTL_CRITICAL_SECTION@@K@ZEA 0000000180024428     MSVCRT:thread_safe_statics.obj
 0003:0001b430       ?g_wake_all_condition_variable@@3P6AXPEAU_RTL_CONDITION_VARIABLE@@@ZEA 0000000180024430     MSVCRT:thread_safe_statics.obj
 0003:0001b43c       ?__proc_attached@@3HA      000000018002443c     MSVCRT:dll_dllmain.obj
 0003:0001b450       ?is_initialized_as_dll@@3_NA 0000000180024450     MSVCRT:utility.obj
 0003:0001b451       ?module_local_atexit_table_initialized@@3_NA 0000000180024451     MSVCRT:utility.obj
 0003:0001b458       ?module_local_atexit_table@@3U_onexit_table_t@@A 0000000180024458     MSVCRT:utility.obj
 0003:0001b470       ?module_local_at_quick_exit_table@@3U_onexit_table_t@@A 0000000180024470     MSVCRT:utility.obj
